:10800000FEDF07EA000000000000000000000000A2
:108010000000000000000000000000000000000060
:108020000000000000000000000000000000000050
:108030000000000000000000000000000000000040
:108040000000000000000000000000000000000030
:02000004001FDB
:020000040020DA
:1000000002D3A0E3A60000EBFEFFFFEA001080E5AC
:100010001EFF2FE1B010C0E11EFF2FE10010C0E570
:100020001EFF2FE1000090E51EFF2FE10E00A0E172
:100030001EFF2FE110FF2FE11EFF2FE110402DE9E1
:1000400008009FE5F6FFFFEB1040BDE81EFF2FE123
:100050005450213F10402DE91C009FE5F0FFFFEBBD
:10006000010010E3FBFFFF0A10009FE5ECFFFFEB30
:100070001040BDE8FF0000E21EFF2FE15450213F79
:100080004050213F10402DE90C009FE5E4FFFFEBBD
:100090001040BDE8010000E21EFF2FE15450213F57
:1000A00010402DE90040A0E11C009FE5DCFFFFEBC4
:1000B000200010E3FBFFFF0A0410A0E10C009FE505
:1000C000D1FFFFEB1040BDE81EFF2FE15450213F50
:1000D0004050213F10402DE910009FE5D0FFFFEB7D
:1000E000010C10E3FBFFFF1A1040BDE81EFF2FE1DB
:1000F0005450213F70402DE90050A0E12040A0E382
:10010000044044E23504A0E10F0000E2090050E39E
:100110003700808230008092E0FFFFEB000054E364
:10012000F6FFFF1A2000A0E37040BDE8DBFFFFEA06
:1001300010402DE9EEFFFFEB0D00A0E3D7FFFFEB32
:100140000A00A0E31040BDE8D4FFFFEA10402DE90B
:100150000110A0E3D4009FE5ABFFFFEB0010A0E38C
:10016000CC009FE5A8FFFFEB0010A0E3C4009FE5D3
:10017000A5FFFFEB0310A0E3BC009FE5A2FFFFEB90
:100180000010A0E3B4009FE59FFFFFEB0010A0E389
:100190009C009FE59CFFFFEBC610A0E3A0009FE53D
:1001A00099FFFFEB9C109FE59C009FE596FFFFEBFE
:1001B00098009FE59AFFFFEB3F1AC0E3121A81E314
:1001C00088009FE590FFFFEB0010A0E380009FE513
:1001D0008DFFFFEB0040A0E30400A0E1014084E2BA
:1001E00094FFFFEB960054E3FAFFFF1A0319A0E314
:1001F00060009FE584FFFFEB0040A0E30400A0E166
:10020000014084E28BFFFFEB960054E3FAFFFF1AF4
:100210000010A0E33C009FE57BFFFFEB0310A0E391
:1002200010009FE578FFFFEB1040BDE81EFF2FE1B7
:100230000450213F4450213F6050213F4C50213F0A
:100240005050213F4850213F0E0100006850213F8F
:100250000400203F9400203F9800203F10402DE9EB
:100260001C409FE5F918A0E30400A0E166FFFFEB46
:100270000400A0E10C109FE563FFFFEB1040BDE818
:100280001EFF2FE108B4003F0002F90010402DE9E5
:1002900008009FE562FFFFEB1040BDE81EFF2FE165
:1002A00020B4003FF0472DE90080A0E3A6FFFFEB5C
:1002B00040029FE59DFFFFEB5BFFFFEB9BFFFFEB2A
:1002C0004900A0E375FFFFEB4800A0E373FFFFEBDD
:1002D0004500A0E371FFFFEB5800A0E36FFFFFEBC9
:1002E0000D00A0E36DFFFFEB0A00A0E30890A0E182
:1002F0000860A0E10850A0E10870A0E10840A0E17A
:1003000066FFFFEB52FFFFEB3A0050E32B00000AC1
:100310000D0050E30A00501301A0A00300A0A01399
:100320002900000A2030C0E3470053E35000000AD0
:10033000013044E2140053E303F19F97F0FFFFEA1A
:10034000B0032000B003200050042000500420001F
:10035000500420005004200030042000F803200046
:10036000D4032000D4032000D4032000D4032000B1
:10037000C80320009403200094032000940320006D
:100380009403200094032000940320009403200091
:1003900094032000390050E3070040820992A0E155
:1003A0000F0000E2150054E3099080E14500000AC7
:1003B00027FFFFEB3A0050E3014084E2D3FFFF1A2E
:1003C0000140A0E3CEFFFFEA0662A0E10040A0E307
:1003D000CBFFFFEA390050E3070040820662A0E14C
:1003E0000F0000E2066080E10668A0E12668A0E157
:1003F000014084E2C2FFFFEA390050E30700408277
:100400000552A0E10F0000E2055080E1FF5005E237
:10041000010055E32700000A0E40A033B8FFFF3A61
:10042000020055E30940A0030040A013B4FFFFEA17
:10043000390050E3070040820552A0E10F0000E2BE
:10044000055080E1FF5005E20840A0E3ACFFFFEA61
:10045000390050E3070040820772A0E10F0000E27C
:10046000077080E10778A0E1277886E1014084E207
:10047000A3FFFFEA0D00A0E308FFFFEB2D00A0E3C0
:1004800006FFFFEB2D00A0E304FFFFEB0D00A0E350
:1004900002FFFFEB0A00A0E300FFFFEB0A00A0E36E
:1004A000FEFEFFEB0209A0E3E1FEFFEB0A00A0E184
:1004B000F047BDE81EFF2FE10800A0E11BFFFFEBA6
:1004C0000040A0E38EFFFFEA693829E02334A0E171
:1004D000FF3CC3E3699423E00700A0E1088087E0C4
:1004E0000910A0E1C8FEFFEB088089E0047087E2F4
:0C04F0000E40A0E382FFFFEA78563412B1
:040000030000800079
:00000001FF
